:100000000428FF3FFF3FFF3F031383129F01831626
:100010008501860187018801890183128501860196
:10002000870188018901A0013830A1000830A200B1
:100030001030A300A401A501A601A7012008860095
:10004000013088000230FB00FF30FA00FB0B29284A
:100050002C28FA0B292826284A30FA00FA0B2E28D9
:1000600021088600023088000230FB00FF30FA00D1
:10007000FB0B3B283E28FA0B3B2838284A30FA0075
:10008000FA0B402822088600043088000230FB006A
:10009000FF30FA00FB0B4D285028FA0B4D284A2858
:1000A0004A30FA00FA0B52282308860008308800EC
:1000B0000230FB00FF30FA00FB0B5F286228FA0BCE
:1000C0005F285C284A30FA00FA0B6428240886006E
:1000D000103088000230FB00FF30FA00FB0B712863
:1000E0007428FA0B71286E284A30FA00FA0B762829
:1000F00025088600203088000230FB00FF30FA001F
:10010000FB0B83288628FA0B832880284A30FA00C4
:10011000FA0B882826088600403088000230FB0051
:10012000FF30FA00FB0B95289828FA0B95289228A7
:100130004A30FA00FA0B9A28270886008030880097
:100140000230FB00FF30FA00FB0BA728AA28FA0BAD
:10015000A728A4284A30FA00FA0BAC28A80A2808D5
:100160001F3A031DDC29A801A9012908073C031C2B
:100170007729AA012A08073C031C7129AB01FF302B
:10018000AC008030013AF00080302C067002031C75
:100190000A29FF30AD008030013AF00080302D0692
:1001A0007002031C04292C082907F0000730700591
:1001B000F2007208AE002D082A07F0000730700523
:1001C000F3007308AF002030F0007208700784005D
:1001D0000008F2000130F00073080319F328F00D55
:1001E0007010FF3FED287208F00573080319FC2812
:1001F000F00CF013FF3FF6287008AB072D08013A0A
:1002000003190429AD0ACB282C08013A03190A293D
:10021000AC0AC1282030F0002908700784000008CB
:10022000F2000130F0002A0803191A29F00D7010AD
:10023000FF3F14297208F0052A0803192329F00C3E
:10024000F013FF3F1D290930F400DE217008AB07D1
:100250002B08033A031934292B080C3A03193429C3
:100260002B080D3A031D4F293030F0002908700784
:10027000F3000130F2002A0803194229F20D72102E
:10028000FF3F3C29730884000008F0007208F00466
:100290007308840073088400700880006B29303074
:1002A000F00029087007F3000130F0002A08031954
:1002B0005D29F00D7010FF3F57297009F200730897
:1002C00084000008F0007208F005730884007308C9
:1002D0008400700880002A08073A03197129AA0AC5
:1002E000BA282908073A03197729A90AB528A901C4
:1002F0002908073C031CDC29AA012A08073C031C27
:10030000D6292030F00029087007F3003030F000C3
:100310002908700784000008F2000130F0002A0864
:1003200003199629F00D7010FF3F90297008F2050F
:100330002A0803199F29F20CF213FF3F992972082A
:10034000003A031DBB290130F0002A080319AC292B
:10035000F00D7010FF3FA6297009F20073088400A9
:100360000008F0007208F005730884007308840028
:1003700070088000D0290130F2002A080319C4292E
:10038000F20D7210FF3FBE29730884000008F000D0
:100390007208F004730884007308840070088000F9
:1003A0002A08073A0319D629AA0A7D292908073AF3
:1003B0000319DC29A90A78291E28DD2903138312D1
:1003C0007008F100F0010830FC007108F40C03180B
:1003D000ED29FC0BE629F10100340310F229F40C9D
:1003E0000318F107F10CF00CFC0BEF290800FF3F9C
:02400E003A3F37
:00000001FF
